:1007C6004D4B49542D342076332E300D004F4B0DB2
:0107D6000022
:07082C0075A61E75A6E1226E
:040003007FC87E0034
:10000700EF4E601712082C7D737C00ED1D70011CEC
:0B001700ED4C70F7EF1F70E81E80E555
:0100220022BB
:0307B5001207B870
:0E07B800C2A0120003D2A07F2C7E0102000717
:10071600EFC394614006EFD39466400CEFC3944157
:10072600400BEFD394465005EF24098001EF540F98
:02073600FF22A0
:09081300000000000000000022BA
:05083A00D2B202081318
:03081C0012083A85
:05081F00C2B202081343
:0E07D700D2B3D2B2C2B3120813C2B2D2B3224E
:0A080900C2B3D2B2120813D2B32218
:1006F2007E01EF339200A20092B3EF25E0FF1208D1
:100702001C0EBE09EDD2B312083AA2B3920012082F
:030712001FA20023
:0107150022C1
:10073800E4FF7E0112083AA2B39200EF25E0FFA27F
:1007480000E433420712081F0EBE09E8D2B31208AC
:010758001C84
:01075900227D
:1006CB00E4FF7E0112083AA2B39200EF25E0FFA2ED
:1006DB0000E433420712081F0EBE09E8C2B312082A
:0606EB003A12081FD2B311
:0106F10022E6
:100674001207D77FA01206F2E4FF1206F2E4FDEDA2
:1006840025E02422F8E6FEEEFF1206F2ED25E02432
:0F06940022F808E6FF1206F20DBD08E30208097E
:1005A4001207D77FA01206F2E4FF1206F21208091E
:1005B4001208131207D77FA11206F2E4FC1206CB2D
:1005C400AD07EDFEEC25E02422F8A606087600BC73
:1005D4000707120738AD0780051206CBAD07EC25D7
:1005E400E02422F8E6FE08E6FFEDFBEB4FFFEC25E6
:1005F400E02422F8A60608A6070CBC08C0020809D5
:08082400300AFDC20A8F99227F
:10060400BF3A0FE4F556D20B7E247832E4F608DEC6
:10061400FC22300B2AEF640D6003BFFF0C743225FB
:1006240056F8A607C20BD20922EFC394204010E566
:0F06340056C39423500974322556F8A60705566D
:010643002294
:030023000206A32F
:0D06A300C0E0C0D075D000C000C006C00788
:1006B000309906C299D20A8007AF99C298120604EF
:0B06C000D007D006D000D0D0D0E03230
:100779008F80EEFF30E104D2A68002C2A6EF30E0FE
:0607890003D2A722C2A763
:01078F002247
:0C07E500D3EF9458EE9402400122D3227E
:1007A300C2A07F647E00120007D2A07F5F7E00029A
:0207B30000073D
:07083300C2A1C2A3C2A4226E
:05083F00D2A4D2A322A7
:10064400D2A1C2A3C2A4C2A07F647E00120007127A
:10065400082C30A20E30A50BE590655760F1E590AB
:10066400F460ECD2A0D2A4D2A37F647E000200077F
:10079000759852758920758DFD438780D28ED2ACB5
:0307A000D2AF22B3
:1005330012082C30096AC209E532C394314012E52E
:1005430032D39438500BAF32120716EF14F55B8099
:10055300087BFF7A0779C68044E55BD3940740089C
:1005630074FFF55CF55D800EE55B25E02422F8E67B
:10057300F55C08E6F55DE55DF47003E55CF4602089
:10058300E55D455C7007E55BD394005013AF5DAE4A
:100593005C1207791206447BFF7A0779D31200882D
:0105A3002235
:10038200AF908F57BFFF0512053380F4E557244124
:10039200602024E0602124F0602224F8602324FC01
:1003A200602424FE6025146027247F702875580776
:1003B20080267558068021755805801C7558048062
:1003C200177558038012755802800D755801800800
:1003D200E4F55880037558FFE558B4FF0874FFF53B
:1003E20059F55A800EE55825E02422F8E6F5590819
:1003F200E6F55AE55AF47003E559F4601AE55A45F0
:10040200597007E558D39400500DAF5AAE591207F0
:1004120079120644120003E59065576003020382D5
:0A0422007FD07E071200070203825C
:1004BA0020970512082C80F81207B51207B8120700
:1004CA00B87B10782274FFF608DBFC900000E4FB8E
:1004DA0012082C20970512000380042090F222EBC8
:1004EA0025E02422F8A68308A682AF82AE831207EB
:1004FA00791208331207A3A3AF82AE831207E5501D
:10050A00063097F012000312083FA3A3A3A30BEB34
:10051A00D394075009AF82AE831207E540B2C2A056
:08052A0030900512082C80F846
:0105320022A6
:0C07F100D2A01206747FF47E0102000703
:10075A007F207E031200071205A4120790120003DD
:0F076A002097061204BA1207F11207B502038294
:030000000207FDF7
:0C07FD00787FE4F6D8FD75817102075A80
:10002600E56D2461F8E6056D22785E300702786199
:10003600E475F00112048402042C2000EB7F2ED21A
:10004600008018EF540F2490D43440D4FF30040BB2
:10005600EF24BFB41A0050032461FFE56E60021559
:100066006E0571E5717002057030070D785EE475F6
:10007600F001120484EF0204720208247403D2070A
:100086008003E4C207F56D8B5E8A5F8960E4F56ED6
:10009600F570F571E56E60077F2012006180F575D9
:1000A6006FFFC201C200C202C203C205C206C20875
:1000B60012002FFF700D3007057F00120072AF711E
:1000C600AE7022B4255FC2D5C20412002FFF24D021
:1000D600B40A00501A75F00A786E30D50508B6FFD6
:1000E6000106C6A426F620D5047002D20380D924C0
:1000F600CFB41A00EF5004C2E5D204020272D20154
:1001060080C6D20080C0D20280BCD2D580BAD205C9
:1001160080B47F201200612002077401B56E004092
:10012600F1120026FF12006102009AD208D2068060
:1001360095120026FB120026FA120026F94A4B7089
:100146000679437A037BFF20022EE56E602A7E0045
:100156008E8275830012044560060EEE656F70F0A0
:10016600C2D5EBC0E0EAC0E0E9C0E0EE1202B9D0C9
:10017600E0F9D0E0FAD0E0FB12042CFF60AAEBC055
:10018600E0EAC0E0E9C0E0120061D0E02401F9D065
:10019600E03400FAD0E0FBE56F0460DCD56FD9806F
:1001A600877BFF7A0279B5D202809C79108002792A
:1001B60008C206C2088008D2D5790A8004790AC224
:1001C600D5E56F047002F56FE4FAFDFEFF12002616
:1001D600FC7B08200113120026FD7B1030000A125A
:1001E6000026FE120026FF7B20EC3382D592D550E6
:1001F60013C3E43000069FFFE49EFEE42001039D46
:10020600FDE49CFCE4CBF8C201EC700CCFCECDCC67
:10021600E824F8F870F38017C3EF33FFEE33FEEDF2
:1002260033FDEC33FCEB33FB994002FB0FD8E9EBD3
:10023600300105F8D0E0C448B201C0E00AEC4D4EEA
:100246004F78207B0070C2EAB56F0040BCC0E01258
:1002560002BBD0F0D0E0200104C4C0E0C4B201C0AB
:10026600F012004AD0F0D5F0EB02009A1204940185
:10027600375301B15801084C01044201B54F01BD85
:0F0286004401BD49011D4301C35501A74601A70E
:100295004501A747036350010C2D01102E01332B97
:1002A500011423013120034C2A00CC480000012B06
:1002B5003F3F3F00790AA2D5200314300509B91044
:1002C500020404B9080104A2D52006025001042045
:1002D50002689202B56E005034C0E07F20300319E9
:1002E5007F30A20272067205500F120312C202C2BB
:1002F50006C205C2087F30800F300503E9C0E01251
:100305000061300503D0E0F9D0E0B56ECC300517BB
:100315007F30B9100C1200617F583004077F788058
:1003250003B908031200613002057F2D0200617FC9
:10033500202008F87F2B2006F322920280CF286E1A
:10034500756C6C2900D2011200263001F8C20178C3
:100355006E30D50108F60200CC2D504349581200E5
:10036500262403B405004001E490035E9312005275
:0D037500743A120052D203756E040201B1F9
:10042C00BB010689828A83E0225002E722BBFE02CE
:09043C00E32289828A83E4932201
:10044500BB010CE58229F582E5833AF583E022506C
:1004550006E92582F8E622BBFE06E92582F8E222B6
:0D046500E58229F582E5833AF583E49322D0
:10047200BB010689828A83F0225002F722BBFE0169
:02048200F32263
:10048400FAE6FB0808E6F925F0F618E6CA3AF62279
:10049400D083D082F8E4937012740193700DA3A3F7
:1004A40093F8740193F5828883E47374029368600B
:0604B400EFA3A3A380DF0B
:00000001FF
